:100000000C941C010C94970A0C94700A0C944401F3
:100010000C9444010C94630C0C9444010C94350C26
:100020000C94A80C0C9444010C9444010C944401CD
:100030000C9444010C9444010C9444010C9444012C
:100040000C94260A0C9444010C94E40A0C94BE0A05
:100050000C9444010C9444010C9444010C9444010C
:100060000C94160B0C9444016803180172681880F4
:10007000234020034C69676874734F4E04034F4E4E
:10008000042020202020BE5004B03B805F50046834
:100090003B0205680576380A01285004683B282F82
:1000A0006805183802004F680576380A00295004A0
:1000B000683B212650046832101E50046832111F1C
:1000C000C004BF1103696804800200EE8003680168
:1000D000EA1804FF0200E16804C00200AEC0036831
:1000E00001AA681880234020032041555820492F39
:1000F0005004032020042020202020E968188023B9
:10010000402003425420417564696F040320200499
:100110002020202020F368188023402003555342DC
:10012000617564696F04032020042020202020A131
:1001300068188023402003464D20626E64203104FD
:10014000032020042020202020C168188023402084
:10015000034C6F6E677761766504032020042020CE
:10016000202020BC681880234020034D2E2057619A
:1001700076652004032020042020202020D5681844
:100180008023402003464D20426E64203304032028
:1001900020042020202020E36818802340200346EC
:1001A0004D20626E64203204032020042020202091
:1001B00020C26805183803004E6805763803002011
:1001C000180A68390209003F0001017768051838EC
:1001D00001004C6804BF0201D00000000024002789
:1001E000002A0000000000250028002B000000006D
:1001F00008000201000003040700000000000000E6
:100200000000000000230026002900040404040468
:1002100004040402020202020203030303030301B3
:10022000020408102040800102040810200102048A
:1002300008102000800DF71211241FBECFEFD8E068
:10024000DEBFCDBF24E0A2E7B1E001C01D92A53B17
:10025000B207E1F711E0A0E0B1E0E4E0F9E202C0AA
:1002600005900D92A237B107D9F711E0CBE1D1E0AB
:1002700004C02197FE010E943A13CA31D107C9F781
:100280000E945F0E0C9475140C940000833081F072
:1002900028F4813099F08230A9F008958730A9F0D0
:1002A0008830C9F08430B1F4809180008F7D03C024
:1002B000809180008F7780938000089584B58F7738
:1002C00084BD089584B58F7DFBCF8091B0008F777A
:1002D0008093B00008958091B0008F7DF9CFCF93C7
:1002E000DF93282F30E0F901E351FE4F8491F901AB
:1002F000E15EFD4FD491F901E55FFD4FC491CC2340
:10030000A1F081110E944601EC2FF0E0EE0FFF1FDB
:10031000EF5FFD4FA591B491EC91ED2381E090E06A
:1003200009F480E0DF91CF91089580E090E0FACF6A
:100330001F93CF93DF93282F30E0F901E351FE4F55
:100340008491F901E15EFD4FD491F901E55FFD4F24
:10035000C491CC23A9F0162F81110E944601EC2FE5
:10036000F0E0EE0FFF1FED51FE4FA591B4918FB756
:10037000F894EC91111108C0D095DE23DC938FBF67
:10038000DF91CF911F910895DE2BF8CFCF93DF93AC
:1003900090E0FC01E15EFD4F2491855F9D4FFC01E3
:1003A00084918823C9F090E0880F991FFC01E752DF
:1003B000FE4FA591B491FC01ED51FE4FC591D49132
:1003C00061110DC09FB7F8948C91209582238C9376
:1003D0008881282328839FBFDF91CF9108956230C1
:1003E00051F49FB7F8943C91822F809583238C938E
:1003F000E8812E2BEFCF8FB7F894EC912E2B2C9316
:100400008FBFEACF3FB7F89480913A0290913B02B8
:10041000A0913C02B0913D0226B5A89B05C02F3F9C
:1004200019F00196A11DB11D3FBFBA2FA92F982F1A
:100430008827BC01CD01620F711D811D911D42E015
:10044000660F771F881F991F4A95D1F708952FB718
:10045000F894609136027091370280913802909141
:1004600039022FBF08950895089508950895AF9211
:10047000BF92CF92DF92EF92FF920F931F93CF9391
:10048000DF936C017B018B01040F151FEB015E01F3
:10049000AE18BF08C017D10759F06991D601ED9188
:1004A000FC910190F081E02DC6010995892B79F727
:1004B000C501DF91CF911F910F91FF90EF90DF90D9
:1004C000CF90BF90AF900895FC01538D448D252FA0
:1004D00030E0842F90E0821B930B541710F0CF96DE
:1004E000089501970895FC01918D828D981761F010
:1004F000A28DAE0FBF2FB11D5D968C91928D9F5F27
:100500009F73928F90E008958FEF9FEF0895FC0105
:10051000918D828D981731F0828DE80FF11D858DB8
:1005200090E008958FEF9FEF0895FC01918D228D4B
:10053000892F90E0805C9F4F821B91098F739927D0
:1005400008958EE392E00E94950221E0892B09F440
:1005500020E0822F089580E090E0892B29F00E940E
:10056000A10281110C9400000895FC01A48DA80F34
:10057000B92FB11DA35ABF4F2C91848D90E00196E5
:100580008F739927848FA689B7892C93A089B18905
:100590008C91837080648C93938D848D981306C0A6
:1005A0000288F389E02D80818F7D80830895EF920A
:1005B000FF920F931F93CF93DF93EC0181E0888F1D
:1005C0009B8D8C8D98131AC0E889F989808185FFED
:1005D00015C09FB7F894EE89FF896083E889F9898F
:1005E00080818370806480839FBF81E090E0DF9191
:1005F000CF911F910F91FF90EF900895F62E0B8DE4
:1006000010E00F5F1F4F0F731127E02E8C8D8E119E
:100610000CC00FB607FCFACFE889F989808185FF05
:10062000F5CFCE010E94B502F1CFEB8DEC0FFD2F7F
:10063000F11DE35AFF4FF0829FB7F8940B8FEA89C0
:10064000FB8980818062CFCFCF93DF93EC01888DCF
:100650008823B9F0AA89BB89E889F9898C9185FD3D
:1006600003C0808186FD0DC00FB607FCF7CF8C91CB
:1006700085FFF2CF808185FFEDCFCE010E94B502CC
:10068000E9CFDF91CF9108952091BA01260F33274A
:10069000331F21323105ECF420910902FC0190E076
:1006A00080E0243069F082E00895A091BA012191A0
:1006B000AC0146565E4FA40FB52FB11D2C93019689
:1006C000861798F38091BA01680F6093BA0180E0B1
:1006D000089581E008951092090281E08093080254
:1006E0001092E30161E082E10E94980161E083E100
:1006F0000E949801E9EBF0E080818E7F8083808109
:100700008D7F808388E48093B80085E48093BC006B
:100710000895CF93DF9391E0909399018823B9F0E6
:10072000C091B800D091BA008091BC008A7B8093C0
:10073000BC0060E082E10E94980160E083E10E94D9
:1007400098010E946B03D093BA00C093B800DF9168
:10075000CF9108950895E091E2018091E101E817B9
:1007600030F4F0E0E758FE4F808190E008958FEF7D
:100770009FEF08959091E2018091E1012FEF3FEF0B
:10078000981748F4E92FF0E0E758FE4F208130E059
:100790009F5F9093E201C90108958091E1019091DA
:1007A000E201891B990B0895CF92DF92EF92FF929D
:1007B0000F931F93CF93DF937C01CB018A0120918C
:1007C0000F02222389F0EB016B01C40ED51ECC155C
:1007D000DD0569F06991D701ED91FC910190F081FF
:1007E000E02DC7010995F3CF642F0E944403C8018F
:1007F000DF91CF911F910F91FF90EF90DF90CF90FD
:100800000895CF93DF931F92CDB7DEB76983209110
:100810000F022223F9F020913202203258F021E019
:1008200030E0FC013383228390E080E00F90DF9181
:10083000CF91089580911002E82FF0E0EF5EFD4F18
:10084000998190838F5F809310028093320281E0C0
:1008500090E0ECCF61E0CE0101960E944403F7CF17
:1008600090E080E00895FC018481958122813381AC
:100870002817390771F0860F971F608171810E94D8
:1008800026130680F781E02DE80FF91F808190E0A4
:1008900008958FEF9FEF0895FC0184819581228157
:1008A00033812817390741F0860F971F60817181C6
:1008B0000E942613958384830895FC01462F22818C
:1008C0003381C9010196608171810E942613648180
:1008D00075818617970781F0A681B781A20FB31F94
:1008E0004C93828193810196608171810E942613CD
:1008F0009383828380E008958FEF0895EF92FF92B3
:100900000F931F93CF93DF937C01062F10E0B80164
:1009100081EA94E00E945D04D0E0C0E0C017D107F6
:1009200058F4F701EC0FFD1F649170E081EA94E048
:100930000E945D042196F2CFDF91CF911F910F911C
:10094000FF90EF900895CF93DF93FC01C281D38194
:1009500084819581C817D907C9F0A681B781A80FEE
:10096000B91F2C910196608171810E942613C817CE
:10097000D90739F095838483822F90E0DF91CF915E
:1009800008951582148213821282F6CF8FEF9FEFA3
:10099000F5CFFC0160817181848195819B01281BC9
:1009A000390B82819381820F931F0E942613089531
:1009B000DC01ED91FC910190F081E02D0994809192
:1009C00078018823B9F080917701882399F06CE051
:1009D00080EC91E00E947E0467E089EB91E00E9448
:1009E0007E0467E082EB91E00E947E0461E08AE091
:1009F0000C94980160E08AE00E94980167E08CEC1A
:100A000091E00C947E048F929F92AF92BF92CF920E
:100A1000DF92EF92FF924B015C010E9402026B0198
:100A20007C0124E0C21AD108E108F1080E94020208
:100A30006C197D098E099F09681579058A059B0542
:100A4000A8F3FF90EF90DF90CF90BF90AF909F9072
:100A50008F9008958091DA03882319F060E00C9458
:100A600098012D980895882349F08091DA0388230E
:100A700019F061E00C9498012D9A08950C942A05C0
:100A8000CF93DF93EC018091DB03823019F481E096
:100A90000E943305299ABE0190E080E00E94030580
:100AA00029988091DB03823031F40E942A05DF917E
:100AB000CF910C942A05DF91CF9108958F929F9248
:100AC000AF92BF92CF92DF92EF92FF92CF934B0102
:100AD0005C01219A8FEF88169806A806B806C1F423
:100AE000219A80E093E20E94400560EC78E080E08B
:100AF00090E00E94030580E392E0CF91FF90EF9099
:100B0000DF90CF90BF90AF909F908F900C94400556
:100B100080E093E20E94400560E871E180E090E0AF
:100B20000E940305C0E2C12CD12CE12C90E8F92EE3
:100B3000D501C4018C219D21AE21BF21892B8A2B97
:100B40008B2B89F080E392E00E94400560E976E01B
:100B500080E090E00E940305F694E794D794C79450
:100B6000C15031F7C8CF80E392E00E94400560E3B6
:100B700072E080E090E0EECFCF9329E534E0F90118
:100B800001900020E9F79F012A553440C091540498
:100B900033274C2F50E0BA0161507109261B370BE7
:100BA00030934F0420934E04682F70E0675A7B4FB8
:100BB00086E191E00E94651480911601803219F45B
:100BC00086E880931601CB5FC0931101EC2FF0E013
:100BD000319620E090E0A92FB0E0A05FBE4F4C918D
:100BE00024279F5FC917B8F7E05FFE4F208360910D
:100BF000110170E06E5F7F4F89EA94E00E945D040E
:100C0000C0E02C2F30E08091110190E00196821716
:100C100093075CF0205F3E4FF901608170E089EA44
:100C200094E00E945D04CF5FECCFCF91089585EDF5
:100C30008093BC0080910B0290910C02A0910D0258
:100C4000B0910E020796A11DB11D23E0B695A795A0
:100C5000979587952A95D1F72091BC0024FD03C074
:100C600010920902089540910B0250910C0260917C
:100C70000D0270910E02452B462B472B69F300970E
:100C8000A105B10541F02AE22A95F1F700C00197CC
:100C9000A109B109E1CF80910A020C948903FC01FA
:100CA00086819781009711F00C94DC1308951F93AF
:100CB000CF93DF93EC01162F0E941013181739F011
:100CC000612FCE01DF91CF911F910C941813DF910A
:100CD000CF911F9108950C9410138BE090E00E9427
:100CE0006B06282F30E030930B0120930A018330EC
:100CF000A1F028F4813041F0823059F00895843019
:100D000081F0853091F008956AE180E391E00C94E0
:100D10007E046AE188E991E0FACF6AE18EE791E02A
:100D2000F6CF6AE184E691E0F2CF6AE18AE491E0ED
:100D3000EECFCF93DF9390E080E00E946B06C82F48
:100D4000D0E0D0930901C09308018AE090E00E94AE
:100D50006B06282F30E0309307012093060121977E
:100D600039F4833019F180F48130B1F08230D1F060
:100D70008AE090E00E946B0690E0909307018093D8
:100D80000601DF91CF9108958430A1F0853081F77D
:100D90006AE18AE491E003C06AE180E391E00E94A5
:100DA0007E04E6CF6AE188E991E0F9CF6AE18EE757
:100DB00091E0F5CF6AE184E691E0F1CF90E080E048
:100DC0000E946B06282F30E0309305012093040128
:100DD0008330D1F028F4813041F0823061F0089501
:100DE0008630D0F0873011F10895109277010E947B
:100DF000DF040C946D06109277010E94DF046AE113
:100E000086E191E00C947E04109277010E94DF0449
:100E10006AE18CEF90E0F6CF6AE182EE90E00E940A
:100E20007E0481E0809377010C94DF0410927701B7
:100E3000FBCF8F929F92AF92BF92CF92DF92EF92B1
:100E4000FF920F931F93CF93DF93CDB7DEB76897D1
:100E50000FB6F894DEBF0FBECDBF7C01FC01008150
:100E6000C280D38016810E942702809072019090E8
:100E70007301A0907401B09075019B01AC01281919
:100E800039094A095B0949015A0130E1831637E201
:100E90009306A104B10468F060937201709373012A
:100EA000809374019093750165E088E690E00E945C
:100EB0007E0445E050E06DED70E0C7010E94031331
:100EC000892B29F466E087ED90E00E947E0446E0DD
:100ED00050E061ED70E0C7010E940313892B19F403
:100EE00081E0809378018091340281110AC066E02C
:100EF00083ED91E00E947E040E94DE0681E08093F3
:100F0000340245E050E06CEC70E0C7010E9403132E
:100F1000892B29F466E086EC90E00E947E0445E08F
:100F200050E060EC70E0C7010E940313892B11F4BC
:100F30000E94DE06003809F055C24FEBC41255C2BC
:100F400058E1D51252C261E081E10E94980180917E
:100F50007601811105C00E94DE0681E08093760152
:100F600068960FB6F894DEBF0FBECDBFDF91CF916C
:100F70001F910F91FF90EF90DF90CF90BF90AF90B7
:100F80009F908F900895153009F487C0163041F76F
:100F900066E08AE990E00E947E04809177018823D0
:100FA00009F4B4C080917801882309F4AFC067E0E8
:100FB00083E990E08CC0193009F4E1C008F4ABC0BB
:100FC0001A3009F45DC165E77AE88EE491E61B30DA
:100FD00009F428C2C5CF183209F4E8C148F5133224
:100FE00009F4ACC190F41E3009F0BACF61E08AE098
:100FF0000E9498018CE00E946F01892B09F483C143
:1010000060E08CE00E949801A3C0163209F4C1C1CF
:10101000173209F0A5CF80917701882321F08091C4
:101020007801811156C06FE070EF8EE491E6FAC14D
:101030001C3209F488C158F4193209F4CEC16FE5A5
:1010400070EA8EE491E61B3209F4ECC189CF1D32BF
:1010500009F47EC11E3409F083CF60E08AE068960F
:101060000FB6F894DEBF0FBECDBFDF91CF911F91B9
:101070000F91FF90EF90DF90CF90BF90AF909F9037
:101080008F900C94980166E08AEB90E00E947E04B9
:1010900067ED78E28EE491E6C5C166E084EB90E00E
:1010A0000E947E0467E578EA8EE491E6BBC166E0C3
:1010B0008EEA90E00E947E048091770167E08823A9
:1010C000E1F0809178018823C1F087EA90E00E94E6
:1010D0007E0468960FB6F894DEBF0FBECDBFDF91D9
:1010E000CF911F910F91FF90EF90DF90CF90BF9025
:1010F000AF909F908F900C94DF0480EA90E00E9464
:101100007E0467EB78E48EE491E68CC167E378ECCB
:101110008EE491E687C166E08DE890E00E947E044F
:101120006FEA70E58EE491E60E945E05809104010D
:1011300090910501019685309105F4F49093050195
:10114000809304016091040190E080E00E945706C2
:1011500068960FB6F894DEBF0FBECDBFDF91CF917A
:101160001F910F91FF90EF90DF90CF90BF90AF90C5
:101170009F908F900C94DE0681E090E0DFCF90E0AE
:1011800080E00E946B06E82EF12CF0920901E092BB
:10119000080181E0E816F104B9F56FE470EB8EE424
:1011A00091E60E945E0585E090E0909303018093B4
:1011B000020180910A0190910B0101968630910500
:1011C000F4F490930B0180930A0160910A018BE083
:1011D00090E00E94570668960FB6F894DEBF0FBEE7
:1011E000CDBFDF91CF911F910F91FF90EF90DF90D6
:1011F000CF90BF90AF909F908F900C946D06F0921F
:101200000B01E0920A01E1CF90E080E00E946B06C2
:1012100090E09093090180930801029709F0A0CE15
:1012200080910601909107010196909307018093A8
:10123000060120910201309103012817390734F487
:1012400081E090E090930701809306016091060190
:101250008AE090E00E94570668960FB6F894DEBFC9
:101260000FBECDBFDF91CF911F910F91FF90EF90F7
:10127000DF90CF90BF90AF909F908F900C94990685
:10128000809100019091010101968630910564F5ED
:1012900090930101809300016091000188E290E049
:1012A0000E94570688E290E00E946B0690E09093BF
:1012B00001018093000128E1E6E3F1E0DE011196EF
:1012C00001900D922A95E1F7880F991F880F991FB9
:1012D000E1E0F0E0EC0FFD1F8E0F9F1FFC0160812D
:1012E0007181828193819EC0109201011092000150
:1012F000D3CF66E087E890E00E947E0465E97AE655
:101300008EE491E68FC061E08CE00E9498016AE172
:101310008DE690E068960FB6F894DEBF0FBECDBFA5
:10132000DF91CF911F910F91FF90EF90DF90CF90C1
:10133000BF90AF909F908F900C947E046FE170EE01
:101340008EE491E66FC065EC7AE38EE491E66AC0C4
:1013500061E090E080E00E94570661E08AE090E062
:101360000E94570661E08BE090E00E94570660E023
:101370008EE190E00E94570660E088E290E00E94D3
:10138000570660E08CE890E00E9457060E94DE0657
:1013900063CF80917701882321F0809178018111BA
:1013A00098CE6FE870E78EE491E63CC062E090E092
:1013B00080E068960FB6F894DEBF0FBECDBFDF9118
:1013C000CF911F910F91FF90EF90DF90CF90BF9042
:1013D000AF909F908F900C9457066FE470EB8EE463
:1013E00091E620C0003C09F0BBCDF1E3DF12B8CD9F
:1013F00061E085E00E9498011C3009F47ACF08F082
:10140000EACD173009F453CE08F0D5CD143009F4E5
:101410003ACE08F0B8CD67E978E68EE491E613306D
:1014200009F09ECD68960FB6F894DEBF0FBECDBF13
:10143000DF91CF911F910F91FF90EF90DF90CF90B0
:10144000BF90AF909F908F900C945E051F920F926B
:101450000FB60F9211242F933F938F939F93AF93C7
:10146000BF938091360290913702A0913802B091DB
:1014700039023091350223E0230F2D3758F50196BC
:10148000A11DB11D2093350280933602909337023F
:10149000A0933802B093390280913A0290913B02B6
:1014A000A0913C02B0913D020196A11DB11D809317
:1014B0003A0290933B02A0933C02B0933D02BF914D
:1014C000AF919F918F913F912F910F900FBE0F90F1
:1014D0001F90189526E8230F0296A11DB11DD2CFAB
:1014E0001F920F920FB60F9211242F933F934F9399
:1014F0005F936F937F938F939F93AF93BF93EF937C
:10150000FF93E0910E01F0910F010995FF91EF918A
:10151000BF91AF919F918F917F916F915F914F910B
:101520003F912F910F900FBE0F901F9018951F9213
:101530000F920FB60F9211242F933F934F935F9307
:101540006F937F938F939F93AF93BF93EF93FF938B
:10155000E0910C01F0910D010995FF91EF91BF9180
:10156000AF919F918F917F916F915F914F913F913B
:101570002F910F900FBE0F901F9018951F920F92F2
:101580000FB60F9211242F933F934F935F936F9356
:101590007F938F939F93AF93BF93EF93FF938EE3CC
:1015A00092E00E94B502FF91EF91BF91AF919F91A0
:1015B0008F917F916F915F914F913F912F910F90FC
:1015C0000FBE0F901F9018951F920F920FB60F929B
:1015D00011242F938F939F93EF93FF93E0914E02EB
:1015E000F0914F028081E0915402F091550282FD0A
:1015F0001BC09081809157028F5F8F73209158029A
:10160000821741F0E0915702F0E0E25CFD4F958FC8
:1016100080935702FF91EF919F918F912F910F909F
:101620000FBE0F901F9018958081F4CF1F920F92DC
:101630000FB60F9211242F933F934F935F936F93A5
:101640007F938F939F93AF93BF93EF93FF9380917B
:10165000B900887F803609F44AC0F0F5883209F471
:10166000A7C018F5803109F49BC0B8F4882309F4A9
:10167000F9C0883009F494C0FF91EF91BF91AF9108
:101680009F918F917F916F915F914F913F912F919A
:101690000F900FBE0F901F901895883109F488C0E5
:1016A000803251F78093070214C0803409F49DC042
:1016B00040F48033B9F38833F9F68093070285EC60
:1016C000B0C0803509F485C0883509F496C08834E7
:1016D00099F60E941706D0CF883909F48CC038F5E6
:1016E000883729F050F4883611F0803729F683E0E6
:1016F000809309021092DC0157C0883809F47BC03E
:10170000803919F0803809F0B7CF8091DC01803240
:1017100008F071C0E091DC0181E08E0F8093DC0164
:101720008091BB00F0E0E454FE4F80833DC0803BDD
:1017300039F0E0F4803A09F479C0883A09F09CCF96
:1017400084E0809309021092BB011092BA01E091EB
:10175000DF01F091E00109958091BA0181110FC07C
:1017600081E08093BA0110929A0109C0803C09F48B
:10177000A6CF883C09F4A3CF883B09F07DCFE09148
:10178000BB0181E08E0F8093BB01F0E0E656FE4F77
:1017900080818093BB009091BB018091BA0129C0E8
:1017A0008091E4018093BB0085EC8093BC0064CF02
:1017B0009091060280910502981758F5E091060273
:1017C00081E08E0F80930602F0E0EB51FE4F8081A6
:1017D000E9CFE091060281E08E0F809306028091AE
:1017E000BB00F0E0EB51FE4F8083909106028091A8
:1017F00005029817C8F285E8D8CFE091060281E08B
:101800008E0F809306028091BB00F0E0EB51FE4FFB
:1018100080838091080281115CCF81E08093E30195
:1018200084EA8093BC001092090226CF85EC809355
:10183000BC00109209028091DC01803230F4E0910A
:10184000DC01F0E0E454FE4F10826091DC0170E0B6
:10185000E091DD01F091DE018CEB91E009951092B1
:10186000DC010ACF1092070234CF1F920F920FB6FD
:101870000F9211242F933F934F935F936F937F9316
:101880008F939F93AF93BF93EF93FF9381E08093E8
:10189000330260E08DE00E949801E1EBF0E080818E
:1018A000887F8083FF91EF91BF91AF919F918F913E
:1018B0007F916F915F914F913F912F910F900FBE4C
:1018C0000F901F9018951F920F920FB60F92112430
:1018D0002F933F934F935F936F937F938F939F9338
:1018E000AF93BF93EF93FF9380E00E946F01019746
:1018F000D9F481E00E946F010197B1F48091B100A9
:1019000087608093B100FF91EF91BF91AF919F915C
:101910008F917F916F915F914F913F912F910F9098
:101920000FBE0F901F90189580E00E946F01892BC9
:1019300051F781E00E946F01019729F7109233025D
:1019400061E08DE00E9498018091B100887FD9CF3D
:101950001F920F920FB60F9211242F933F934F9324
:101960005F936F937F938F939F93AF93BF93CF9327
:10197000EF93FF93E091F102F091F202C081809128
:10198000F302C8238091F4029091F502019649F088
:101990008091F4029091F50201969093F502809364
:1019A000F4028091EF0281111DC0C1116EC08091BF
:1019B000F4029091F502813A910578F01092F802C4
:1019C0008091F4029091F5029093FB028093FA02C9
:1019D00081E08093F9028093EF021092F502109259
:1019E000F40253C08091EF028130A9F4CC2309F4B2
:1019F0004CC0E091F9028E0F8093F9028091F402BD
:101A00009091F502F0E0EE0FFF1FE151FD4F94873A
:101A1000838782E0E0CF8091EF02823009F04FC0EF
:101A2000C11122C0E091F90281E0E03768F08093B3
:101A3000F80283E08093EF02E091F602F091F70262
:101A4000309759F20995C9CF8E0F8093F902809192
:101A5000F4029091F502F0E0EE0FFF1FE151FD4F0F
:101A60009487838781E0B7CF8091F4029091F5024B
:101A7000813A910550F083E08093EF02E091F60205
:101A8000F091F702309709F009958091DB038130DE
:101A900021F4C11180E00E943305FF91EF91CF91B5
:101AA000BF91AF919F918F917F916F915F914F9176
:101AB0003F912F910F900FBE0F901F90189580911E
:101AC000EF02833011F7C111E0CF87CF0F931F933F
:101AD000CF93DF93EC018B01798368831D821C8295
:101AE0001B821A82CB010E9440139F838E83A80120
:101AF00070E060E0DF91CF911F910F910C946E1414
:101B0000CF93DF93EEE3F2E01382128288EE93E04C
:101B1000A0E0B0E084839583A683B78322E531E01B
:101B20003183208325EC30E03587248724EC30E0B6
:101B30003787268720EC30E0318B208B21EC30E09A
:101B4000338B228B22EC30E0358B248B26EC30E07B
:101B5000378B268B118E128E138E148EEBEDF2E0E6
:101B60001382128284839583A683B78384E691E0EF
:101B7000918380830E9427026093EB027093EC02B2
:101B80008093ED029093EE020E9427026093E70299
:101B90007093E8028093E9029093EA0260E870E0B3
:101BA00089E994E00E94660D60E470E081EA94E0C7
:101BB0000E94660D60E470E089EA94E00E94660D80
:101BC000EFEEF2E0F0930304E0930204118281E06F
:101BD000848389E290E09383828350981092DA03A1
:101BE000CFE0D4E01CAA0E9427026093EB0270931E
:101BF000EC028093ED029093EE020E942702609324
:101C0000E7027093E8028093E9029093EA02198652
:101C10001A861B8618861F821E821D8262E080E063
:101C20000E94C60161E084E00E94C60161E084E098
:101C30000E949801E0EBF0E010821092B1008DE973
:101C40008093B300808182608083E0E7F0E0808150
:101C500082608083E8E6F0E0808184608083EDE646
:101C6000F0E080818160808319821A8280ED97E0A4
:101C70009AAF89AF88EE93E09CAF8BAF88EC90E091
:101C80009EAF8DAF82E08093550410924F04109266
:101C90004E048BE080935404109256041092570423
:101CA000109258040E9427026093500470935104CC
:101CB0008093520490935304DF91CF9108957894C8
:101CC00084B5826084BD84B5816084BD85B5826041
:101CD00085BD85B5816085BD80916E0081608093F2
:101CE0006E0010928100809181008260809381005B
:101CF000809181008160809381008091800081606B
:101D0000809380008091B10084608093B1008091C5
:101D1000B00081608093B00080917A0084608093ED
:101D20007A0080917A00826080937A0080917A00B4
:101D3000816080937A0080917A00806880937A0035
:101D40001092C10061E085E00E94C60161E086E07A
:101D50000E94C60160E08AE00E94C60161E08BE05B
:101D60000E94C60161E08CE00E94C60162E084E14D
:101D70000E94C60161E08DE00E94C601E0914E0222
:101D8000F0914F0282E08083E0914A02F0914B0291
:101D90001082E0914C02F0914D0280E1808310921C
:101DA0005602E0915202F091530286E08083E09166
:101DB0005002F0915102808180618083E091500255
:101DC000F0915102808188608083E0915002F0910F
:101DD0005102808180688083E0915002F09151022D
:101DE00080818F7D808361E085E00E949801109260
:101DF000E2011092E10110921002109232020E9450
:101E00006B0384E392E09093E0018093DF0185E32C
:101E100092E09093DE018093DD0181E080930F02D8
:101E20008FE2809331026FE78BED92E00E94010414
:101E3000C0913202C13208F091C00E9402026B01CF
:101E40007C0180910902811164C082E080930902C3
:101E500081E0809308028FEF8093070210920602C0
:101E6000C0930502A1E1B2E0E5EEF1E080E0C81325
:101E700023C11092E4018091E4018E658093E40116
:101E80008091E301813009F01BC11092E3010E94AF
:101E900002026B017C018091E4018093BB00809180
:101EA0000B0290910C02A0910D02B0910E02892BB1
:101EB0008A2B8B2B99F00E94020200910B02109149
:101EC0000C0220910D0230910E026C197D098E09D1
:101ED0009F090617170728073907E0F18091BC0012
:101EE00083FDD9CF85EC8093BC000E9402026B0178
:101EF0007C0180910902823009F4E4C080910702DC
:101F00008F3F61F180910702803241F18091070299
:101F100025C080910B0290910C02A0910D02B0910E
:101F20000E02892B8A2B8B2B09F48BCF0E94020285
:101F300000910B0210910C0220910D0230910E02C3
:101F40006C197D098E099F0906171707280739079D
:101F500008F077CF80910A020E9489031092100244
:101F60001092320210920F028EE392E090931304CB
:101F700080931204E0914E02F0914F0292E0908320
:101F8000E0914A02F0914B021082E0914C02F091F4
:101F90004D028FEC808310925602E0915202F09134
:101FA000530286E28083E0915002F09151028081D9
:101FB00080618083E0915002F091510280818860BD
:101FC0008083E0915002F09151028081806880838B
:101FD000E0915002F091510280818F7D80832CED41
:101FE00035E0309349042093480428EE33E03093E1
:101FF0004B0420934A0428EC30E030934D042093A6
:102000004C049093550489E197E0909347048093A2
:10201000460461E08DE00E94C60192E0292E312C39
:10202000EE24E394F12C34E0C32ED12C80913402C1
:1020300081112FC00E9402024B015C0188EE482EE4
:1020400083E0582E612C712C0E94020268197909D4
:102050008A099B09683E734081059105A8F321E038
:10206000421A51086108710888EE880E83E0981EB4
:10207000A11CB11C411451046104710429F766E0EC
:1020800083ED91E00E947E040E94DE06B1E0B093F1
:102090003402E0911404F0911504E830F105B0F534
:1020A000EC5AFF4E0C943A1384103F1155117811DD
:1020B000A111B611CA11EB119D9191938F5FD7CEEB
:1020C00085EE11CF80910B0290910C02A0910D0230
:1020D000B0910E02892B8A2B8B2B09F40ACF0E9418
:1020E000020200910B0210910C0220910D0230911E
:1020F0000E026C197D098E099F090617170728071C
:10210000390708F0F6CE26CF10925604809133029C
:102110008823E1F089EA94E00E94C90418161906A0
:10212000ACF489EA94E00E94A304EC0180E00E94F0
:102130006F01019731F4B12CA12CC331D10508F402
:1021400070C1BE0189EA94E00E944C04809112049F
:1021500090911304DC01ED91FC910084F185E02D58
:102160000995892B81F08091120490911304DC0170
:10217000ED91FC910284F385E02D0995BC0189E97C
:1021800094E00E945D0480911604909117048230BF
:10219000910509F49BC108F058C1009709F463C187
:1021A000019709F475C1809133028823C9F181EA4E
:1021B00094E00E94C9041816190694F50E9427029B
:1021C0000091E7021091E8022091E9023091EA02C1
:1021D000601B710B820B930B6A30710581059105B1
:1021E000F8F081EA94E00E94A304EC0180E00E94F0
:1021F0006F01019731F4B12CA12CC132D1050CF43F
:10220000E2C1BE0181EA94E00E944C040E942702D0
:102210006093E7027093E8028093E9029093EA02E8
:1022200080911004882371F00E94270260E084E00E
:102230000E94980170E060E0809112049091130474
:102240000E94D8040E94270261347F4181059105D4
:1022500048F08BE00E946F01019721F460E08BE071
:102260000E94980180E090E0892B09F4DFCE0E9463
:10227000A102882309F4DACE0E940000D7CE109282
:1022800058041092570480E00E94BC053092150457
:10229000209214040E94270260935004709351040A
:1022A000809352049093530431CF0E9427020091EF
:1022B0005004109151042091520430915304AB0109
:1022C000BC01401B510B620B730B80914804909131
:1022D0004904B0E0A0E0481759076A077B0708F4F3
:1022E00015CF83E090E090931504809314040ECFF3
:1022F0008091570420914E0430914F0482171306A9
:1023000080F48F5F809357048091580491E0980F78
:10231000909358040E94BC05D0921504C0921404F6
:10232000B9CFA5E0B0E0B0931504A09314041092C7
:10233000580410925704809156048F5F809356047E
:10234000E5CE0E9427020091500410915104209183
:10235000520430915304AB01BC01401B510B620B82
:10236000730B80914C0490914D04B3CF909156041F
:1023700080915504981738F486E090E09093150406
:102380008093140487CFA7E0B0E0B0931504A09326
:10239000140480CF0E942702009150041091510430
:1023A0002091520430915304AB01BC01401B510BEE
:1023B000620B730B80914A0490914B04B0E0A0E053
:1023C000481759076A077B0708F4A0CEF092150456
:1023D000E09214049BCE0E942702009150041091B9
:1023E00051042091520430915304AB01BC01401BB5
:1023F000510B620B730B80914A0490914B04B0E037
:10240000A0E0481759076A077B0708F47FCE1092AF
:10241000580480E00E94BC05109215041092140428
:1024200075CE0091120410911304CA15DB0509F44E
:102430008DCE89EA94E00E94A304BC01C8010E94E9
:10244000D804BFEFAB1ABB0AECCF8330910509F477
:1024500077C061E070E0049709F0A5CE89E994E0C7
:102460000E944C04ABC089E994E00E94C90418168C
:1024700019060CF098CE70E060E089E994E00E94C3
:10248000330480931804F0921704E09216048BCE64
:1024900089E994E00E94C90402970CF484CE61E0BB
:1024A00070E089E994E00E9433048093190483501A
:1024B000823228F4309217042092160474CE61E020
:1024C00070E089E994E00E944C046DCE00911904FB
:1024D00010E05801BFEFAB1ABB0A89E994E00E94F3
:1024E000C904A816B9060CF05ECE712CD0E0C0E08D
:1024F000BE0189E994E00E943304782621960C17E6
:102500001D07B4F7B50189E994E00E9433047816F9
:10251000190689F40E9427026093EB027093EC0283
:102520008093ED029093EE0283E090E09093170485
:102530008093160438CED0921704C092160433CE7E
:1025400080911804982F9F77903521F0982F9F7BCA
:10255000903899F4CFE0D4E09E012F50344021967A
:102560008091190490E0019682179307ECF089E9B5
:1025700094E00E94A3048B87EFCF893759F3982FFB
:102580009D7F983639F38F3329F3883119F3982FCB
:102590009F7D983CF9F26091190470E06E5F7F4F67
:1025A000803B09F05BCFD6CF91E090934304E0915C
:1025B0004604F09147048BE194E0099510921704CA
:1025C00010921604F0CDAC16BD060CF01FCE009193
:1025D00012041091130481EA94E00E94A304BC0148
:1025E000C8010E94D804AFEFAA1ABA0AECCF89EA50
:1025F00094E00E944F0681EA94E00E944F0689E928
:1026000094E00C944F06FB01DC0104C08D91059011
:10261000801921F441505040C8F7881B990B089548
:10262000F999FECF92BD81BDF89A992780B508959A
:10263000262FF999FECF1FBA92BD81BD20BD0FB6DE
:10264000F894FA9AF99A0FBE01960895AA1BBB1B3B
:1026500051E107C0AA1FBB1FA617B70710F0A61BA2
:10266000B70B881F991F5A95A9F780959095BC01C3
:10267000CD010895EE0FFF1F0590F491E02D099410
:102680000F931F93CF93DF938230910510F482E074
:1026900090E0E091B304F091B40430E020E0B0E0C9
:1026A000A0E0309799F42115310509F44AC0281BA0
:1026B000390B24303105D8F58A819B81611571056C
:1026C00089F1FB0193838283FE0111C04081518116
:1026D0000281138148175907E0F04817590799F408
:1026E000109761F012960C93129713961C933296E2
:1026F000CF01DF91CF911F910F9108950093B30403
:102700001093B404F4CF2115310551F0421753074B
:1027100038F0A901DB019A01BD01DF01F801C1CF49
:10272000EF01F9CF9093B4048093B304CDCFFE01B1
:10273000E20FF31F8193919322503109398328834B
:10274000D7CF2091B1043091B204232B41F42091D2
:102750003201309133013093B2042093B1042091BF
:102760003001309131012115310541F42DB73EB7CB
:102770004091340150913501241B350BE091B10497
:10278000F091B204E217F307A0F42E1B3F0B2817B9
:10279000390778F0AC014E5F5F4F2417350748F0DA
:1027A0004E0F5F1F5093B2044093B10481939193F5
:1027B0009FCFF0E0E0E09CCFCF93DF930097E9F06C
:1027C000FC01329713821282A091B304B091B40439
:1027D000ED0130E020E01097A1F420813181820FDB
:1027E000931F2091B1043091B2042817390709F0E2
:1027F00061C0F093B204E093B104DF91CF910895EA
:10280000EA01CE17DF07E8F54A815B819E01411599
:102810005105B1F7E901FB83EA8349915991C40F4E
:10282000D51FEC17FD0761F4808191810296840F1A
:10283000951FE90199838883828193819B838A8391
:10284000F0E0E0E012968D919C9113970097B9F516
:102850002D913C911197CD010296820F931F2091EB
:10286000B1043091B2042817390739F6309751F581
:102870001092B4041092B304B093B204A093B104C4
:10288000BCCFD383C28340815181840F951FC81769
:10289000D90761F44E5F5F4F88819981480F591FB6
:1028A000518340838A819B819383828321153105E3
:1028B00009F0B0CFF093B404E093B3049ECFFD01D0
:1028C000DC01C0CF13821282D7CFFB01DC0102C032
:1028D00001900D9241505040D8F70895DC0101C09D
:1028E0006D9341505040E0F7089511E0CBE1D1E005
:1028F00004C0FE010E943A132196CC31D107C9F7DA
:04290000F894FFCF79
:10290400010001000100010001000100360236024D
:10291400C8008023423200000000000000000000D4
:1029240000000000000000000000000000000000A3
:102934000000B50480007D824E61BD424E613DC2FF
:102944004E61DD224E615DA24E619D624E610000CA
:102954000000D7023702640224039502730287023F
:10296400000000000104D4033004AA03CD03BA0319
:02297400AB03B3
:00000001FF
